:100000000C9424020C9468020C9468020C9468020C
:100010000C9468020C9468020C9468020C946802B8
:100020000C9468020C9468020C94F70C0C94C90DA3
:100030000C9468020C9468020C9468020C94680298
:100040000C9468020C94D3210C9468020C946802FE
:100050000C9468020C94661B0C9468020C94680261
:100060000C9468020C9468020C9468020C94680268
:100070000C9468020C9468020C9468020C94680258
:100080000C9468020C9468020C9468020C94680248
:100090000C9468020C9468020C9468020C94680238
:1000A0000C9468020C9468020C946802360E580E88
:1000B000460F580E460F9D0EC00E460F150F280F07
:1000C000F711F711261226125C127C12AD13AD1334
:1000D0008712AD13371337139E13AD13AD13A71348
:1000E0004413441344134413441344134413441358
:1000F0004413441344134413441344134413441348
:10010000561363136A1371137B1335002B00E00041
:10011000E1003A0000001E00140004001D003B0036
:10012000E2001F001A0016001B003C00297120008D
:100130000700080006003D002A0021000900170002
:100140001900E300A90022000E000A0005000000CB
:10015000AA003E00310000002F000000A8003F0070
:100160000154000030000000AE0023000D001C0010
:1001700013000000AB002400180011001000E7007D
:10018000AC00250015000C00360050002C002600A5
:100190000F001200370051003400270033000B001D
:1001A00038005200E6002E002D002800E5004F0028
:1001B0000000010001000100010001000000010039
:1001C0000100010001000100010001000100010027
:1001D000010001000100010008000700010001000A
:1001E00001000100150009000100010001000100EB
:1001F00017000100010000000100010001000000E3
:1002000001000000010001000100000001000000E9
:10021000010001001C000B001100000001000100A2
:1002200018000D0001000100010001000C000E008B
:10023000010001000100010012000F000100010097
:100240000100010013003300010001000100010062
:1002500001000100010001000000160345007200CA
:1002600067006F0044006F007800200045005A00CE
:10027000000016034500720067006F0044006F0025
:100280007800200045005A00000004030904090218
:100290006D00040100A0FA0904000001030101003F
:1002A000092111010001223F000705810308000A0E
:1002B00009040100010301020009211101000122CA
:1002C0004D000705820308000A090402000103002B
:1002D00000000921110100012236000705830308EF
:1002E000000A0904030001030000000921110100B4
:1002F00001223900070584031000011201100100DA
:10030000000008EDFE0713010001020001050109CC
:1003100006A101050719E029E715002501950875D3
:1003200001810205081901290595057501910295BC
:10033000017503910105071900297715002501951D
:100340007875018102C005010980A10185021601AD
:100350000026B7001A01002AB70075109501810028
:10036000C0050C0901A1018503160100269C021A93
:1003700001002A9C02751095018100C00501090247
:10038000A1010901A100050919012905150025018F
:1003900095057501810295017503810105010930FB
:1003A00009311581257F9502750881060938158167
:1003B000257F950175088106050C0A3802158125EF
:1003C0007F950175088106C0C005010906A10105D8
:1003D0000719E029E71500250195087501810295A7
:1003E0000175088101050819012905950575019117
:1003F000029501750391010507190029FF150025D4
:10040000FF950675088100C0000000000000000094
:10041000000000010204060A0F17202C3A4A5D7101
:10042000879DB3C7DAE9F5FCFFFCF5E9DAC7B39DB0
:1004300087715D4A3A2C20170F0A0604020100005A
:10044000000000000000000011241FBECFEFDAE022
:10045000DEBFCDBF04B603FE24C08091FB019091A6
:10046000FC01A091FD01B091FE018730904BA740A7
:10047000B04BB9F41092FB011092FC011092FD01F7
:100480001092FE0114BE84B7877F84BF88E10FB647
:10049000F89480936000109260000FBEE0E0FFE3EC
:1004A000099511E0A0E0B1E0E4E3F7E402C00590B3
:1004B0000D92A433B107D9F711E0A4E3B1E001C074
:1004C0001D92AB3FB107E1F70E943B0A0C949823C1
:1004D0000C9400001092B9008AE08093B80008954F
:1004E00094EA9093BC009091BC0097FFFCCF909150
:1004F000B900987F983021F0903111F081E0089593
:100500008093BB0084E88093BC008091BC0087FF8F
:10051000FCCF8091B900887F883111F0803471F769
:1005200080E0089584E98093BC008091BC0084FD44
:10053000FCCF08958093BB0084E88093BC00809139
:10054000BC0087FFFCCF9091B900987F81E0983282
:1005500009F480E0089584E88093BC008091BC0099
:1005600087FFFCCF8091BB0008958091010181112C
:1005700015C080E40E9470028093010181110CC0BB
:1005800082E10E949A0280930101811105C08FEFE0
:100590000E949A02809301010E94920284B1807F9E
:1005A00084B985B1807F85B98AB1837F8AB98BB1DF
:1005B000837F8BB93E98469808950E94700480937B
:1005C00001010E94B50280B38C7080BB81B3836F40
:1005D00081BBA5E3B1E0E3E4F1E08EE08E0F119280
:1005E0001D928E13FCCF0C945A04BF92CF92DF92CF
:1005F000EF92FF920F931F93CF93DF9380910101AE
:10060000882379F0809134018F5F809334018111C8
:1006100008C00E94700480930101811102C00E94F1
:10062000020405E311E0C0E0D0E0DD24D39482E0D1
:10063000C82EEE24E394F12CC730D10500F580914B
:100640000101811164C080E40E9470028093010165
:10065000811112C082E10E949A02809301018111EE
:100660000BC0C7010C2E01C0880F0A94EAF78095D1
:100670000E949A02809301010E94920248C0CA30EF
:10068000A1F028F4C83059F0C93061F005C0CC3071
:1006900089F070F0CD3089F0209A289810C0219A06
:1006A00029980DC0229A2A980AC0239A2B9807C02D
:1006B000529A01C0539A5B9802C03E9A469890EABB
:1006C0009A95F1F79FB1799902C082E001C080E06C
:1006D00091709D25982B7C9902C084E001C080E038
:1006E000892B7D9902C038E001C030E0832B7E99D0
:1006F00002C020E101C020E0822B9FB19095991F9C
:100700009927991F9295990F907E892B0FC0809100
:100710000101811149C080E40E94700280930101AF
:10072000882379F1B12C0E9492028B2DF8019081DF
:10073000981719F08083C09200010E94B50221969B
:100740000F5F1F4FCE30D10509F076CF80910001A9
:10075000882361F1815080930001882339F08FE96B
:100760009FE00197F1F700C0000020C0A3E4B1E0D2
:10077000E5E3F1E0CF01825F91919D938E13FCCF71
:1007800015C083E10E949A02809301018111CACFB2
:1007900081E40E947002809301018111C3CF0E9405
:1007A000AB02B82EB094BFCF80E0C0CF0E9400044F
:1007B00081E0DF91CF911F910F91FF90EF90DF903B
:1007C000CF90BF900895E82FF0E0ED5BFE4F808161
:1007D000089508950F931F93CF93DF93C3E4D1E05F
:1007E00010E00C2F025F899190E00E948C1A180F84
:1007F0000C13F9CF812FDF91CF911F910F910895A5
:100800000C94C10456985E9825982D9826982E9899
:1008100027982F988FEF90E090938900809388001D
:1008200090938B0080938A0090938D0080938C002E
:10083000259A2D9A2FEF80E792E02150804090403A
:10084000E1F700C00000269A2E9A2FEF80E792E091
:10085000215080409040E1F700C00000279A2F9A75
:100860002FEF80E792E0215080409040E1F700C0F8
:10087000000025982D982FEF80E792E021508040CE
:100880009040E1F700C0000026982E982FEF80E7F7
:1008900092E0215080409040E1F700C0000027988E
:1008A0002F9856985E9825982D9826982E982798D8
:1008B0002F98089589EA8093800089E080938100D1
:1008C00024982C983F988AB18F748AB96E98479A69
:1008D0008BB1806B8BB9769A0E9402040C94C00491
:1008E00080E2809301018091510181110EC00E942C
:1008F0006A0281E0809351012FEF83ED90E3215054
:1009000080409040E1F700C0000080E40E94700247
:100910008093010181112EC00E949A0280930101EF
:10092000811128C00E949A0280930101811122C086
:100930008FE30E949A028093010181111BC00E94E3
:10094000920280E40E94700280930101811112C022
:100950008CE00E949A028093010181110BC00E94D9
:100960009A0280930101811105C08FE30E949A02CF
:10097000809301010E9492028091010108950895DF
:1009800008956091BD017091BE018091BF01909169
:10099000C0010E94981A56985E9825982D9826981E
:1009A0002E9827982F98813011F4259A2D9A089522
:1009B00081E0089581E008950C94DA0408950F937E
:1009C0001F93CF93DF938C01FC01C081D181CE01B5
:1009D0000E941119BE010E948805EC01B8010E9415
:1009E000DC04882309F48DC0F8018281882309F48E
:1009F0004AC080915D0181111FC0C431F0E5DF075D
:100A000009F051C00E94DE0481E080935D010E94E4
:100A1000301B90935C0180935B0110925401109203
:100A200056011092550110925801109257011092E0
:100A30005A011092590165C080915B0190915C014F
:100A40000E943C1B883C910570F480915401E82F72
:100A5000F0E0EE0FFF1FEB5AFE4FD183C0838F5F94
:100A6000809354014EC0C43880E5D80721F0C538C2
:100A7000D04501F13AC0F8018281882341F01092FB
:100A8000520182E01EC0C438E0E5DE0759F58091CE
:100A90005201811106C086E20E949B1086E20E94EC
:100AA000631182E01CC0C438F0E5DF0741F3C538AC
:100AB000D045D9F4F8018281882331F01092530196
:100AC00080E20E94B2111DC080915301811106C0C5
:100AD00087E20E949B1087E20E94631180E20E94DD
:100AE000B9110FC0C538D04529F381E08093520178
:100AF00080935301C801DF91CF911F910F910C9406
:100B0000D80480E0DF91CF911F910F91089508954F
:100B100096E0799FF001112494E5899FE00DF11D85
:100B20001124E60FF11DEE0FFF1FE65FFE4F8591CA
:100B300094910895880F991FFC01E657F040859124
:100B400094910895880F991FFC01E65FFE4F8591EF
:100B5000949108950F931F93CF93DF93EC01811528
:100B600020E3920750F5C11580E2D80708F0C3C012
:100B7000CB3BD10590F4C83AD10508F06AC0C53A1C
:100B8000D10508F05BC0C430D10508F0D0C1219771
:100B900009F0CAC101E010E00AC2CF3FD10511F04F
:100BA00008F0C5C1C03FD10508F0A2C0CE01805EEB
:100BB0009109089708F4BBC1B7C1C13090E5D907C6
:100BC00009F4A2C020F5C0318FE4D80770F4C11534
:100BD00090E4D90708F094C0C11521E3D20708F0CA
:100BE000A3C1DD278E01106CE2C1C115D04509F00B
:100BF0009BC10E9418148FEF94E32CE08150904029
:100C00002040E1F700C000000E948B1BD0C1C1153D
:100C100097E5D90758F4C03121E5D20708F01CC187
:100C2000C43180E5D80708F475C07EC1CE01905765
:100C30008115904108F078C1DF7073C1C53AD105C4
:100C400009F477C1C63AD10509F076C102E810E48B
:100C5000AEC1C83AD10509F472C1C93AD10509F447
:100C600071C1CA3AD10509F470C1CB3AD10509F472
:100C70006FC1CC3AD10509F46EC1CD3AD10509F462
:100C80006DC1C03BD10509F46CC1CE3AD10509F460
:100C90006BC1CF3AD10509F46AC1C13BD10509F452
:100CA00069C1C23BD10509F468C1C33BD10509F450
:100CB00067C1C43BD10509F466C1C53BD10509F440
:100CC00065C1C63BD10509F464C1C73BD10509F430
:100CD00063C1C83BD10509F462C1C93BD10509F420
:100CE00061C1CA3BD10509F460C100E014E45FC1F1
:100CF0008E0110655CC1CE019F700E94A20558C193
:100D0000DF708E01106A53C18091DA018160809397
:100D1000DA014DC10E94301D811102C00E94161DD2
:100D20000E944D1D90E09093FB018093FA01C23028
:100D300080E5D80721F48091FA01816086C0C43033
:100D400090E5D90721F48091FA0182607EC0C63017
:100D500020E5D20721F48091FA01846076C0C83082
:100D600080E5D80719F48091FA0127C0CA3090E5D0
:100D7000D90721F48091FA01806167C0CC3020E569
:100D8000D20721F48091FA0180625FC0CE3080E505
:100D9000D80721F48091FA01806457C0C03190E5F2
:100DA000D90721F48091FA0180684FC0C23120E553
:100DB000D20729F48091FA018460886046C0C3306C
:100DC00080E5D80721F48091FA018E7F3EC0C530BE
:100DD00090E5D90721F48091FA018D7F36C0C730A4
:100DE00020E5D20721F48091FA018B7F2EC0C93013
:100DF00080E5D80719F48091FA0126C0CB3090E540
:100E0000D90721F48091FA018F7E1FC0CD3020E5F3
:100E1000D20721F48091FA018F7D17C0CF3080E591
:100E2000D80721F48091FA018F7B0FC0C13190E582
:100E3000D90721F48091FA018F7707C0C331D045DB
:100E400031F48091FA018B7F877F8093FA01809142
:100E5000FA010E94511DABC08D2F99278F709927E1
:100E600081309105D9F49E012370332702C0880F89
:100E7000991F2A95E2F79C688E0144E0000F111F2C
:100E80004A95E1F700271370802B912B53E0CC0F8C
:100E9000DD1F5A95E1F7C076DD272FC0823091051E
:100EA00031F4DC2FCC278E01016F106A80C08330B3
:100EB000910569F4CE018370992701E010E002C02A
:100EC000000F111F8A95E2F7C8019C680FC084309B
:100ED0009105B9F4CE018370992701E010E002C0BA
:100EE000000F111F8A95E2F7C8019A6823E0CC0F22
:100EF000DD1F2A95E1F7C07ED7708C010C2B1D2BCE
:100F000056C08530910531F4DC2FCC278E01046F5B
:100F1000106A4DC0069709F04AC0CF71DD27DC2F5B
:100F2000CC278E01106243C000E010E040C08E016B
:100F30003EC001E810E43BC003E810E438C002EE14
:100F400014E435C009EE14E432C00AEE14E42FC0F4
:100F500005EB14E42CC006EB14E429C007EB14E401
:100F600026C00CEC14E423C00DEC14E420C003E80C
:100F700015E41DC00AE815E41AC002E915E417C01B
:100F800004E915E414C001E216E411C003E216E41A
:100F90000EC004E216E40BC005E216E408C006E247
:100FA00016E405C007E216E402C00AE216E4C8012E
:100FB000DF91CF911F910F91089596E0799FF001F5
:100FC000112494E5899FE00DF11D1124E60FF11D18
:100FD000EE0FFF1FE65FFE4F85919491803E9105D5
:100FE000E0F4803C910558F58133910509F46FC018
:100FF00048F48932910509F463C08A32910509F4F5
:101000006DC072C089339105E9F082389105D1F045
:101010008533910509F44DC067C0833E910581F188
:1010200038F4803E9105B9F0823E9105D9F05CC05C
:10103000863E910561F1873E9105A1F155C00E9460
:101040009A0508952091FA0120FD02C021FF4CC0AD
:1010500080EE90E049C08091FA0180FFF9CF89E3EA
:1010600090E042C08091FA0182FF0EC08091FA01A7
:1010700084FF03C080E090E037C083EE90E034C08E
:101080008091FA0182FFF2CF82EE90E02DC0809134
:10109000FA0183FF0BC08091FA0184FDEBCF87EE4C
:1010A00090E022C08091FA0183FFF5CF86EE90E0B8
:1010B0001BC08091FA0185FF07C089E290E014C04F
:1010C0008091FA0185FFF9CF85E390E00DC0809112
:1010D000FA0186FF07C08AE290E006C08091FA011B
:1010E00086FFF9CF81E390E00E94AA050895089554
:1010F0000C94770880916E010895CF93DF9300D010
:101100001F92CDB7DEB79C018091F101843019F5B3
:1011100093E099833B832A839093E9008FEF90912A
:10112000E800815095FD06C095ED9A95F1F7000015
:101130008111F5CF8091E80085FF0DC040E050E0BF
:1011400063E070E0CE0101960E94E70A8091E8001A
:101150008E778093E8000F900F900F90DF91CF91E2
:101160000895CF93DF9300D01F92CDB7DEB72091C3
:10117000F101243021F522E029839B838A8383E0D7
:101180008093E9008FEF9091E800815095FD06C0B3
:1011900095ED9A95F1F700008111F5CF8091E80067
:1011A00085FF0DC040E050E063E070E0CE010196A5
:1011B0000E94E70A8091E8008E778093E8000F9004
:1011C0000F900F90DF91CF9108952091F10124307D
:1011D000F1F422E02093E9002FEF3091E800215054
:1011E00035FD06C035ED3A95F1F700002111F5CF38
:1011F0002091E80025FF0BC040E050E065E070E082
:101200000E94E70A8091E8008E778093E8000895B5
:10121000CF93DF93EC019091F101943009F046C037
:1012200080910C018823D9F080910D018823B9F0B9
:101230009093E9008FEF9091E800815095FD06C0F2
:1012400095E19A95F1F700008111F5CF8091E800C2
:1012500085FF2CC040E050E060E170E017C081E005
:101260008093E9008FEF9091E800815095FD06C0D2
:1012700095ED9A95F1F700008111F5CF8091E80086
:1012800085FF14C040E050E068E070E0CE010E94AD
:10129000E70A8091E8008E778093E80080E1FE0104
:1012A000AEE5B1E001900D928A95E1F7DF91CF9123
:1012B00008958091F001811109C00E947C0C0E9468
:1012C000D90C8091E20084608093E200089510922E
:1012D000F001089508950C94C0210E94211B0E94E2
:1012E000C6210E947F0F0C94780842E061EC81E0F7
:1012F0000E94F60B42E061EC82E00E94F60B42E0B5
:1013000061EC83E00E94F60B42E161EC84E00C9416
:10131000F60B8091F301833009F455C030F481302D
:1013200071F0823009F48EC008958A3009F47AC0D1
:101330008B3009F460C0893009F09CC020C08091D6
:10134000F201813A09F096C08091E800877F80938E
:10135000E8008091F6019091F701892B21F460E17A
:101360008EE591E003C060E080E090E070E00E94D4
:10137000320B8091E8008B778093E800089580918C
:10138000F201813209F076C08091F6019091F70167
:10139000009719F0039709F06DC08091E800877FEE
:1013A0008093E8008091E80082FD05C08091F10102
:1013B0008111F8CF5FC08091F10080936E01809120
:1013C000E8008B7753C08091F201813A09F052C056
:1013D0008091F6019091F701892B09F04BC0809123
:1013E000E800877F8093E8008091E80080FFFCCFD1
:1013F00080910C0136C08091F2018132D9F5809143
:10140000F6019091F701892BA9F58091E800877F7B
:101410008093E8000E942B0C8091F40180930C01D2
:101420000C9418148091F201813221F58091E8002A
:10143000877F8093E8000E942B0C8091F5018093B8
:101440006F0108958091F201813AA1F48091E80042
:10145000877F8093E8008091E80080FFFCCF809137
:101460006F018093F1008091E8008E778093E8000F
:101470000C942B0C089584B7877F84BF88E10FB646
:10148000F89480936000109260000FBE90E080E8B6
:101490000FB6F89480936100909361000FBE0E9494
:1014A000CE0F0E947C0C0E94D90C8091E2008460D7
:1014B0008093E20078940E945F0F0E94D00F82E038
:1014C00091E00E947A0F0E94AE218091F101853057
:1014D00069F40E94E81A8091EF018823B1F30E9419
:1014E000131B882391F30E94D10AEFCF0E94D60FDD
:1014F000ECCF292F332723303105C9F064F4213094
:10150000310581F02230310509F043C08DE690E0CD
:101510002EE832E042C021323105F1F022323105AD
:1015200041F137C082E190E02BEF32E036C09927DD
:101530008130910541F08230910541F0892B49F5C8
:10154000EAE8F2E005C0E2E7F2E002C0EAE5F2E034
:10155000849190E09F0121C06430D8F4E62FF0E040
:10156000EE0FFF1FEE5DFE4F2081318189E090E09C
:1015700014C0643070F470E0FB01EE0FFF1FE65EF4
:10158000FE4F20813181FB01EA5EFE4F808190E0B9
:1015900004C080E090E020E030E0FA013183208355
:1015A000089580E189BD82E189BD09B400FEFDCFC7
:1015B0008091D8008F7D8093D8008091E000826078
:1015C0008093E0008091E00081FDFCCF0895CF92F0
:1015D000DF92EF92FF920F931F93CF93DF93EC0173
:1015E0008B016A010E944A0C811133C0C114D104DD
:1015F00039F0F60180819181081B190BC80FD91FA2
:10160000E12CF12C0115110519F18091E80085FDFF
:1016100016C08091E8008E778093E800C114D10451
:1016200049F0F60180819181E80EF91EF182E08295
:1016300085E00FC00E944A0C882321F30AC08991DB
:101640008093F10001501109FFEFEF1AFF0ADACF82
:1016500080E0DF91CF911F910F91FF90EF90DF908D
:10166000CF9008952091F8013091F901261737079E
:1016700048F06115710539F42091E8002E77209328
:10168000E80001C0B90140E061157105A9F12091A0
:10169000F101222309F443C0253009F442C020910E
:1016A000E80023FD40C02091E80022FD32C02091D7
:1016B000E80020FFE9CF4091F3002091F20030E0F4
:1016C000342BFC01CF016115710559F0283031052B
:1016D00040F481918093F100615071092F5F3F4F79
:1016E000F1CF41E02830310509F040E02091E800D9
:1016F0002E772093E800C8CF4111C9CF0AC080914E
:10170000F101882361F0853061F08091E80083FD6C
:101710000AC08091E80082FFF2CF80E0089582E065
:10172000089583E0089581E008952091F8013091B3
:10173000F9012617370748F06115710539F4209132
:10174000E8002E772093E80001C0B901FC0120E0F9
:101750006115710591F18091F101882309F440C070
:10176000853009F43FC08091E80083FD3DC0809141
:10177000E80082FD2FC08091E80080FFE9CF209132
:10178000F3008091F20090E0922B6115710559F001
:101790008830910540F424912093F10031966150F6
:1017A00071090196F2CF21E0089709F020E08091BD
:1017B000E8008E778093E800CBCF2111CCCF0AC010
:1017C0008091F101882361F0853061F08091E8001B
:1017D00083FD0AC08091E80082FFF2CF80E0089587
:1017E00082E0089583E0089581E00895982F97306E
:1017F00058F59093E900981739F07091EC0020911A
:10180000ED005091F00003C0242F762F50E021FF0F
:1018100019C03091EB003E7F3093EB003091ED002A
:101820003D7F3093ED003091EB0031603093EB0061
:101830007093EC002093ED005093F0002091EE00A7
:1018400027FF07C09F5FD3CF8F708093E90081E0AF
:10185000089580E008958091F20187FF11C0809182
:10186000E80082FD05C08091F1018111F8CF11C01F
:101870008091E8008B770BC08091F101882349F0BB
:101880008091E80080FFF8CF8091E8008E77809308
:10189000E80008952091E4003091E50095E640913C
:1018A000EC00842F817040FF22C08091E80080FD11
:1018B0001CC08091F101882391F0853091F08091D6
:1018C000EB0085FD10C04091E4005091E500421707
:1018D000530729F39A01915011F784E0089582E0AB
:1018E000089583E0089581E0089580E0089540918F
:1018F000E80042FFDECF08950E94EA0C0E94F20C3D
:10190000E0EEF0E0808181608083E8EDF0E08081AE
:101910008F77808319BCA7EDB0E08C918E7F8C937C
:1019200080818F7E80831092F00108950F931F9322
:10193000CF93DF930E94EA0C0E94F20CC8EDD0E036
:1019400088818F77888388818068888388818F7D6C
:10195000888319BC1092F1011092ED011092EF01F1
:101960001092EE0100EE10E0F80180818B7F808301
:1019700088818160888342E060E080E00E94F60B0D
:10198000E1EEF0E080818E7F8083E2EEF0E0808106
:1019900081608083808188608083F80180818E7F70
:1019A0008083888180618883DF91CF911F910F911F
:1019B0000895E8EDF0E080818F7E8083E7EDF0E030
:1019C00080818160808384E082BF81E08093F00128
:1019D0000C94960CE8EDF0E080818E7F808310926D
:1019E000E20008951092DA001092E10008951F922B
:1019F0000F920FB60F9211242F933F934F935F9343
:101A00006F937F938F939F93AF93BF93EF93FF93C6
:101A10008091E10082FF0BC08091E20082FF07C04D
:101A20008091E1008B7F8093E1000E945E0F8091A6
:101A3000DA0080FF1FC08091D80080FF1BC080911A
:101A4000DA008E7F8093DA008091D90080FF0DC08C
:101A500080E189BD82E189BD09B400FEFDCF81E04E
:101A60008093F1010E94590905C019BC1092F1013F
:101A70000E9467098091E10080FF19C08091E20017
:101A800080FF15C08091E2008E7F8093E2008091FC
:101A9000E20080618093E2008091D80080628093B0
:101AA000D80019BC85E08093F1010E946B098091F8
:101AB000E10084FF30C08091E20084FF2CC080E10F
:101AC00089BD82E189BD09B400FEFDCF8091D800B7
:101AD0008F7D8093D8008091E1008F7E8093E1001C
:101AE0008091E2008F7E8093E2008091E20081602D
:101AF0008093E2008091ED01882311F084E007C01B
:101B00008091E30087FD02C081E001C083E0809303
:101B1000F1010E946D098091E10083FF29C080914D
:101B2000E20083FF25C08091E100877F8093E10080
:101B300082E08093F1011092ED018091E1008E7FAF
:101B40008093E1008091E2008E7F8093E20080919B
:101B5000E20080618093E20042E060E080E00E9469
:101B6000F60B8091F00088608093F0000E946A0973
:101B7000FF91EF91BF91AF919F918F917F916F9165
:101B80005F914F913F912F910F900FBE0F901F903B
:101B900018951F920F920FB60F9211242F933F9317
:101BA0004F935F936F937F938F939F93AF93BF9365
:101BB000CF93DF93EF93FF93C091E900CF708091B3
:101BC000EC00D82FD17080FDD0E81092E900809110
:101BD000F000877F8093F00078940E940D0E1092A1
:101BE000E9008091F00088608093F000CD2BCF70E9
:101BF000C093E900FF91EF91DF91CF91BF91AF9139
:101C00009F918F917F916F915F914F913F912F9114
:101C10000F900FBE0F901F9018951F93CF93DF93D7
:101C2000CDB7DEB7AA970FB6F894DEBF0FBECDBF13
:101C3000E2EFF1E088E08E0F9091F10091938E1326
:101C4000FBCF0E9489098091E80083FF1FC180912A
:101C5000F2019091F301492F50E04A30510508F00C
:101C600015C1FA01EA5AFF4F0C944823803881F0DD
:101C7000823809F00BC18091F6018F708093E900E2
:101C80008091EB0085FB882780F91092E90006C05F
:101C90008091EE019091EF01911182609091E800A6
:101CA000977F9093E8008093F1001092F100C8C0F4
:101CB000282F2D7F09F0EAC0882319F0823061F0C7
:101CC000E5C08091F401813009F0E0C0933009F063
:101CD00080E08093EF012BC08091F401811127C037
:101CE0008091F6018F7009F4D1C08093E9002091B2
:101CF000EB0020FF1CC0933021F48091EB00806248
:101D000014C09091EB0090619093EB0021E030E0E3
:101D1000A90102C0440F551F8A95E2F74093EA00DB
:101D20001092EA008091EB0088608093EB001092A3
:101D3000E9008091E800877F86C08111A7C01091DB
:101D4000F4011F778091E3008078812B8093E3007A
:101D50008091E800877F8093E8000E942B0C80919F
:101D6000E80080FFFCCF8091E30080688093E3006F
:101D7000111102C082E001C083E08093F10186C0AE
:101D80008058823008F082C08091F4019091F50172
:101D90008C3D53E0950779F583E08A838AE2898355
:101DA0004FB7F894DE01139620E03EE051E2E32FB6
:101DB000F0E050935700E49120FF03C0E295EF70EC
:101DC0003F5FEF708E2F90E0EA3010F0C79601C0B1
:101DD000C0968D939D932F5F243149F74FBF80911B
:101DE000E800877F8093E8006AE270E0CE01019608
:101DF0000E94320B14C0AE014F5F5F4F6091F6013D
:101E00000E94790ABC01009709F440C09091E80053
:101E1000977F9093E80089819A810E94950B809129
:101E2000E8008B778093E80031C0803879F58091A5
:101E3000E800877F8093E8008091ED018093F100B6
:101E40008091E8008E778093E8000E942B0C1EC0E2
:101E500081111CC09091F4019230C0F48091E8008F
:101E6000877F8093E8009093ED010E942B0C809176
:101E7000ED01811106C08091E30087FD02C081E081
:101E800001C084E08093F1010E9475098091E8000F
:101E900083FF0AC08091E800877F8093E8008091EB
:101EA000EB0080628093EB00AA960FB6F894DEBF39
:101EB0000FBECDBFDF91CF911F9108950895CF93AD
:101EC0008091F1018823A1F0C091E900CF70909139
:101ED000EC00892F817090FD80E8C82B1092E900FA
:101EE0008091E80083FD0E940D0ECF70C093E90041
:101EF000CF91089590937501809374010895E091B6
:101F00007401F0917501309721F00190F081E02D7E
:101F1000099480E00895E0917401F0917501309783
:101F200021F00280F381E02D09940895E09174017D
:101F3000F0917501309721F00480F581E02D09942E
:101F4000089520917201309173018217930771F007
:101F50009093730180937201E0917401F091750187
:101F6000309721F00680F781E02D099408952091A3
:101F70007001309171018217930771F09093710194
:101F800080937001E0917401F0917501309721F018
:101F90000084F185E02D0994089508950C94CD0FE7
:101FA0000E94271B0E94DD020C94E91B9F92AF92B6
:101FB000BF92CF92DF92EF92FF920F931F93CF9336
:101FC000DF9300D000D000D0CDB7DEB70E94F5027D
:101FD0000DE010E0AA24A394B12C902E802F0E9433
:101FE000E303980129583E4F6901F901F080F82672
:101FF000A1F40150110988F78FEF89838A831B822E
:102000000E94301B8160782F9D838C8349815A8187
:102010006B818D810E946D102FC09091DA0191FF2C
:1020200004C08E830E94E9038E8125E030E0A50183
:10203000022E01C0440F0A94EAF7E42E4F21C1F0AA
:1020400029839A828E2191E009F490E09B830E947B
:10205000301B8160782F9D838C8349815A816B81ED
:102060008D810E946D10F6018081E826E08204C017
:1020700021503109E0F6BDCF0E94D01E10917601AB
:102080000E947F0F1817B9F00E947F0F809376018E
:1020900026960FB6F894DEBF0FBECDBFDF91CF916D
:1020A0001F910F91FF90EF90DF90CF90BF90AF9076
:1020B0009F900C94780826960FB6F894DEBF0FBE5A
:1020C000CDBFDF91CF911F910F91FF90EF90DF90E7
:1020D000CF90BF90AF909F900895CF93DF93CDB7EF
:1020E000DEB72B970FB6F894DEBF0FBECDBF4F8380
:1020F000588769877A878B87DE01119686E0FD0114
:1021000011928A95E9F785E0FE01379601900D92CC
:102110008A95E1F749815A816B817C818D819E810D
:102120000E94B6162B960FB6F894DEBF0FBECDBF39
:10213000DF91CF910895CF93882309F4C2C0C82FAF
:10214000823859F40E947F0F81FDBBC089E30E9451
:1021500090190E945D1A89E30CC0833879F40E94BB
:102160007F0F80FDAEC083E50E9490190E945D1A2A
:1021700083E50E94D219CF910C945D1A843859F4EA
:102180000E947F0F82FD9DC087E40E9490190E94EB
:102190005D1A87E4EECF8CEF8C0F813A48F48C2FD8
:1021A0000E94132181118DC08C2F0E949019E3CFC2
:1021B00080E28C0F883048F4C77081E001C0880F3E
:1021C000CA95EAF70E94161AD6CF8BE58C0F83309A
:1021D00078F4C53A29F0C63A31F083E890E005C0BA
:1021E00081E890E002C082E890E0CF910C94A10FCA
:1021F00088E58C0F833108F064C0C83A39F1C93AD8
:1022000041F1CA3A49F1CB3A51F1CC3A59F1CD3AC0
:1022100061F1C03B69F1CE3A71F1CF3A79F1C13B3E
:1022200081F1C23B89F1C33B91F1C43B99F1C53BBC
:10223000A1F1C63BA9F1C73BB1F1C83BB9F1C93B1C
:10224000C1F1CA3BC9F180E090E038C082EE90E075
:1022500035C089EE90E032C08AEE90E02FC085EB69
:1022600090E02CC086EB90E029C087EB90E026C080
:102270008CEC90E023C08DEC90E020C083E891E0EE
:102280001DC08AE891E01AC082E991E017C084E994
:1022900091E014C081E292E011C083E292E00EC0AE
:1022A00084E292E00BC085E292E008C086E292E010
:1022B00005C087E292E002C08AE292E0CF910C94DE
:1022C000B70FCF910895882309F44BC0823859F491
:1022D0000E947F0F81FF45C089E30E9490190E94F0
:1022E0005D1A89E30CC0833871F40E947F0F80FF70
:1022F00038C083E50E9490190E945D1A83E50E9410
:10230000D2190C945D1A843859F40E947F0F82FF11
:1023100028C087E40E9490190E945D1A87E4EFCFDD
:102320009CEF980F913A58F390E2980F983050F440
:10233000877091E001C0990F8A95EAF7892F0E9472
:102340001C1ADFCF9BE5980F933020F480E090E0DB
:102350000C94A10F885A833120F480E090E00C9413
:10236000B70F0895882321F00E94161A0C945D1A65
:102370000895882321F00E941C1A0C945D1A089578
:102380007F928F929F92AF92BF92CF92DF92EF9205
:10239000FF920F931F93CF93DF931F92CDB7DEB7BA
:1023A0007C01C62E772EFC01058102950F701281EB
:1023B00011110E94331A0E948919882379F0112380
:1023C00069F080E28C0D883048F082E00E9472193A
:1023D0000E94891991E0D82ED92601C0D12CE72D71
:1023E000E295EF70F0E0E05AFF4F0C944823872D00
:1023F000807F072D0F70882311F00295007F112335
:1024000089F0002309F490C180E28C0D883020F41B
:10241000802F0E94161A03C0802F0E94261A0E9445
:102420005D1A82C18C2D0E946311002309F495C1AD
:1024300080E28C0D883020F4802F0E941C1A03C08B
:10244000802F0E942C1A0E945D1A87C1972D907FC1
:10245000872D8F70903211F08295807FCC2021F0F3
:10246000F1E0CF16B1F01EC0112349F0002309F4AA
:1024700014C1013009F011C10E94461A6EC1002337
:1024800019F0013009F469C189830E94491A8981D0
:102490000AC1112321F0023008F05FC1FEC0011112
:1024A0005CC101C1112321F0002309F4F6C03CC135
:1024B000002309F4F8C03EC1872D86958695837068
:1024C00090E0009719F0019761F047C1112321F0C6
:1024D0008C2D972D937002C080E090E00E94A10F98
:1024E0003CC1112321F08C2D972D937002C080E008
:1024F00090E00E94B70F31C18C2D112319F00E947A
:10250000D81D02C00E94401E0E94C51E26C1872DF4
:10251000837009F052C0111120C18C2D82958695CF
:102520008770880F880F9C2D9F70892E912CA12C6D
:10253000B12C082E04C0880C991CAA1CBB1C0A9440
:10254000D2F7C4FE14C00FE010E020E030E0B90183
:10255000A80104C0440F551F661F771F8A95D2F744
:10256000CB01BA01609570958095909503C060E0AD
:1025700070E0CB01272D26952695237030E0223080
:10258000310569F02330310589F0682979298A29D4
:102590009B292130310571F00E94FE17DEC06829A9
:1025A00079298A299B290E941A18D7C00E94FE17F0
:1025B000C501B4010E94E217D0C0112319F0872D84
:1025C000817001C08695882309F4C7C08C2D82953F
:1025D00086958770880F880F9C2D9F70892E912C6F
:1025E000A12CB12C082E04C0880C991CAA1CBB1C61
:1025F0000A94D2F7C4FE14C00FE010E020E030E0EF
:10260000B901A80104C0440F551F661F771F8A95A2
:10261000D2F7CB01BA01609570958095909503C073
:1026200060E070E0CB01272D269526952370422F80
:1026300050E04230510569F04330510589F0682976
:1026400079298A299B294130510571F00E94D818B7
:1026500084C0682979298A299B290E94F4187DC0A1
:102660000E94D818C501B4010E94BC1876C08C2DF8
:1026700090E0FC01E05EF109E531F10508F050C0A1
:10268000E059FF4F0C9448230C2D0F70872D8F714C
:10269000112331F00E945518802F0E94B2115DC0A5
:1026A0000E947618802F0E94B91157C0112339F06B
:1026B000011153C0872D8F710E949B184EC00230AC
:1026C00008F04BC0F7CF112339F0872D8F710E948E
:1026D000551843C01123C9F3872D8F710E947618B6
:1026E0003CC0112329F0872D8F710E94401835C0FE
:1026F0000E94361832C0112351F0172D1F71812FFF
:102700000E94551863E0812F0E94691926C081E05C
:102710000E947219023008F182E00E9472191DC0F5
:10272000112331F0002389F28C2D0E949B1015C0DB
:10273000002391F28C2D0E9463110FC0472D4F7022
:102740006C2DC7010E94BF040E945A1706C0472D76
:102750004F706C2DC7010E948705DD20F9F00E94A3
:10276000651980FD1BC0F70112820E945F190E944B
:102770005518C7010E94DD130E945F190F90DF9169
:10278000CF911F910F91FF90EF90DF90CF90BF906E
:10279000AF909F908F907F900C9476180F90DF9160
:1027A000CF911F910F91FF90EF90DF90CF90BF904E
:1027B000AF909F908F907F9008950F931F93CF932A
:1027C000DF93EC01888199812B813C81232BB9F027
:1027D0009F3F11F48F3F99F0CE010E94DF048823C0
:1027E00071F0688179818A810E945B198C010E9455
:1027F00010190E94D717B801CE010E94C011DF91B5
:10280000CF911F910F9108950E94331A0E94431A8D
:102810000E94081A0E945D1A0E94761F0E94C51E1F
:1028200080E090E00E94A10F80E090E00C94B70F50
:102830000E94231A0C9404140E945019292F2295E7
:102840002F7030E02C3031054CF42A3031056CF417
:102850002250310922303105A8F407C02C3031054F
:1028600069F02F30310551F00DC0803F69F018F448
:10287000803E40F409C0843F29F406C093FB8827BA
:1028800080F9089580E0089581E00895CF93DF9363
:1028900000D000D01F92CDB7DEB70F900F900F90F1
:1028A0000F900F90DF91CF910895CF93DF9300D0D9
:1028B00000D000D0CDB7DEB726960FB6F894DEBFB5
:1028C0000FBECDBFDF91CF9108951F93CF93DF93BC
:1028D000C091850116E080918601C81799F0D0E07B
:1028E0001C9FF0011D9FF00D1124E957FE4F408100
:1028F000518162817381848195810E945514219652
:10290000C770E9CFDF91CF911F9108954091B70132
:102910005091B8016091B9017091BA018091BB01E9
:102920009091BC010C9455148091BC0182958F70DC
:1029300009F054C08091B901882309F44FC08091F7
:102940008501A09186016091B7017091B801409115
:10295000BA015091BB01B6E08A1709F43FC090E07C
:1029600041155105C1F17F3F11F46F3FA1F1B89FAF
:10297000F001B99FF00D1124E957FE4F2181721328
:102980002AC02081621327C02281211124C0238103
:1029900034812417350710F421503109241B350BDD
:1029A000283C3105C0F42091BC012F702061209398
:1029B000BC0126E0289FF001299FF00D1124E45767
:1029C000FE4F80818F708061808387EB91E00E9451
:1029D000DD130C94651401968770BECF0895CF92D5
:1029E000DF92EF92FF920F931F93CF93DF93CDB7B8
:1029F000DEB762970FB6F894DEBF0FBECDBF8C0175
:102A000085E0F801DE011D9601900D928A95E1F7AF
:102A1000D8014C9111965C91119712966C91129776
:102A20001396CD90DC9014973091B7017091B80156
:102A30008091BA019091BB01009709F46BC17F3F6F
:102A400019F43F3F09F466C1E090B901EE2009F4A2
:102A5000C0C02091BC01C816D90628F0F601E81BB9
:102A6000F90BCF0104C0809590958C0D9D1DFF241E
:102A7000F394883C910578F0F12C207F09F0C6C0D2
:102A80007C2DD98AC88A89890E94461487EB91E0F7
:102A90000E94DD13B1C0822F807F09F046C07513FC
:102AA00014C0341312C0611110C02F702061209324
:102AB000BC010E94861487EB91E00E94DD13809197
:102AC000BC01D80115968C932EC0CD2819F15F3F1B
:102AD00011F44F3FF9F0F62E61111CC08091850171
:102AE0002091860136E0821709F45AC090E0389FA1
:102AF000F001399FF00D1124E957FE4F71815713F2
:102B000006C07081471303C07281711103C0019622
:102B10008770E9CFF62E662309F418C18091BC01B5
:102B200081608093BC01F12C11C1751308C034136E
:102B300006C0611104C08091BC01D801C3C04D879B
:102B40005E878D859E856A8B0E941C146A89882306
:102B5000E1F16623D1F12091BC01822F82958F7023
:102B600090E0029774F08091B7019091B801988736
:102B70008F831986DB86CA862C87CE0107960E9432
:102B8000DD1386E0F801A7EBB1E001900D928A9584
:102B9000E1F70E9494140E948614FF24F394D6C097
:102BA0004D875E878D859E850E945019292F22951D
:102BB0002F7030E0223031050CF0BCC09F7009F05E
:102BC000B6C0805E883008F4C1C0C8010E94DD1321
:102BD000E4CFC816D90608F453C0F601E81BF90B78
:102BE000CF01883C910508F450C0F12C7C2DD98A86
:102BF000C88A89890E944614E7EBF1E086E0DF018C
:102C00001D928A95E9F70E948614A0C0751314C01E
:102C1000341312C0611110C08091BC01F80185838A
:102C2000C8010E94DD1386E0E7EBF1E0DF011D92B1
:102C30008A95E9F7FE2C8AC04D875E878D859E8533
:102C40006A8B0E941C146A89882309F4BECF66230C
:102C500009F4BBCF2091BC01822F82958F7090E048
:102C600002970CF48ECF8091B7019091B8019A83AE
:102C700089831B82DD82CC822E83CE0101967FCF99
:102C8000809590958C0D9D1DACCFF62E662309F492
:102C90009CCF75132EC034132CC02091BC0120FD95
:102CA0001FC0822F82958F70D9F0D80115962C9372
:102CB00015978F3049F08F5F982F9295907F822FD4
:102CC0008F70892B15968C93C8010E94DD1386E0C6
:102CD000F801A7EBB1E001900D928A95E1F793CF4F
:102CE00086E0F801A7EBB1E001900D928A95E1F73B
:102CF0002DC04D875E878D859E850E941C14811195
:102D000040CF8091BC0181608093BC01C8010E94CA
:102D1000DD131CC0662309F458CF4D875E878D856F
:102D20009E850E941C14882309F44FCF2ACF81115D
:102D300048CF0CC0243031050CF047CF9F7009F408
:102D400040CFF8019581907F09F03BCF8F2D62969F
:102D50000FB6F894DEBF0FBECDBFDF91CF911F91AC
:102D60000F91FF90EF90DF90CF9008951F93CF9336
:102D7000DF93CDB7DEB72C970FB6F894DEBF0FBE4A
:102D8000CDBF4F83588769877A878B879C87CE0111
:102D900007960E94EF14882369F08F8198852A8511
:102DA0003B85232BF1F19F3F09F063C08F3F09F072
:102DB00060C037C086E0FE013796DE0111960190B3
:102DC0000D928A95E1F76F817885EA85FB853097CA
:102DD00041F17F3F11F46F3F21F12091860130E0F6
:102DE000C9010196877099274091850150E08417A9
:102DF000950709F447C069837A83FD83EC8396E0E5
:102E0000929FD001939FB00D1124A957BE4FFE0190
:102E1000319601900D929A95E1F7809386010E9478
:102E2000651416E080918501909186018917C1F1A2
:102E3000189FC001112489579E4F0E94EF148823C8
:102E400079F1E09185011E9FF0011124E957FE4FB1
:102E50004081518162817381848195810E945514E2
:102E60008091850190E00196877099278093850174
:102E7000D9CF4F81588569857A858B859C850E943D
:102E80005514CFCF0E94181410928601109285011C
:102E9000E7EBF1E086E0DF011D928A95E9F7C1CF0B
:102EA0002C960FB6F894DEBF0FBECDBFDF91CF9149
:102EB0001F910895EF92FF920F931F93CF93DF938B
:102EC0008C01009709F46CC0F12CEE24E394E80126
:102ED0002196F8018491843740F4843008F051C081
:102EE000813081F0823019F15BC0853709F444C02C
:102EF000A8F19CE7980F903708F052C08F770E9496
:102F0000631141C00E5F1F4FFE01C49180E28C0F20
:102F1000883048F4C7708E2D01C0880FCA95EAF733
:102F20000E94361A14C08C2F0E949B102DC00E5F79
:102F30001F4FFE01C49180E28C0F883058F4C77097
:102F40008E2D01C0880FCA95EAF70E943C1A0E9494
:102F50005D1A1AC08C2F0E94631116C00E5F1F4F9E
:102F6000FE01C491CC2381F08FE99FE00197F1F736
:102F700000C00000C150F6CF0E5F1F4FFE01F4905D
:102F800003C00E949B108E018F2D882309F49FCFD0
:102F9000EFE9FFE03197F1F700C000008150F5CF75
:102FA000DF91CF911F910F91FF90EF9008950895B9
:102FB0006093C1017093C2018093C3019093C401D7
:102FC0000C9404140F931F930091C1011091C2013E
:102FD0002091C3013091C401DC01CB01802B912BE6
:102FE000A22BB32B8093C1019093C201A093C30184
:102FF000B093C4011F910F910C9404140F931F936D
:103000000091C1011091C2012091C3013091C4010E
:10301000DC01CB0180239123A223B3238093C10140
:103020009093C201A093C301B093C4011F910F916B
:103030000C9404140F931F930091C1011091C201CD
:103040002091C3013091C401DC01CB01802791277D
:10305000A227B3278093C1019093C201A093C3011B
:10306000B093C4011F910F910C9404141092BD01F0
:103070001092BE011092BF011092C0010C94041472
:1030800041E050E060E070E004C0440F551F661F4F
:10309000771F8A95D2F74093BD015093BE0160938C
:1030A000BF017093C0010C94041441E050E060E053
:1030B00070E004C0440F551F661F771F8A95D2F732
:1030C0008091BD019091BE01A091BF01B091C0015E
:1030D000482B592B6A2B7B2B4093BD015093BE018B
:1030E0006093BF017093C0010C94041441E050E060
:1030F00060E070E004C0440F551F661F771F8A957B
:10310000D2F740955095609570958091BD01909152
:10311000BE01A091BF01B091C001482359236A2389
:103120007B234093BD015093BE016093BF01709318
:10313000C0010C94041441E050E060E070E004C071
:10314000440F551F661F771F8A95D2F78091BD01E6
:103150009091BE01A091BF01B091C00148275927AD
:103160006A277B274093BD015093BE016093BF0146
:103170007093C0010C9404140F931F930091BD0130
:103180001091BE012091BF013091C001DC01CB0143
:10319000802B912BA22BB32B8093BD019093BE016A
:1031A000A093BF01B093C0011F910F910C94041420
:1031B0000F931F930091BD011091BE012091BF019B
:1031C0003091C001DC01CB0180239123A223B323E2
:1031D0008093BD019093BE01A093BF01B093C00145
:1031E0001F910F910C9404140F931F930091BD0134
:1031F0001091BE012091BF013091C001DC01CB01D3
:1032000080279127A227B3278093BD019093BE0109
:10321000A093BF01B093C0011F910F910C940414AF
:103220000895CF92DF92EF92FF920F931F93CF9367
:10323000DF938C01C090C101D090C201E090C30126
:10324000F090C4018091BD019091BE01A091BF0199
:10325000B091C001C82AD92AEA2AFB2ACFE1D0E0DE
:10326000D701C6010C2E04C0B695A79597958795F2
:103270000A94D2F780FF06C0B8018C2F0E94DD07A8
:10328000019721F4219760F780E001C08C2FDF9136
:10329000CF911F910F91FF90EF90DF90CF90089505
:1032A000CF93DF93EC010E941119BE010E94DD074C
:1032B000DF91CF910895CB010E945019089580911C
:1032C000C50185958595859508958091C50187707F
:1032D000089598E0899F90011124262B2093C50121
:1032E0000C9455182091C501809582238093C501C7
:1032F000982F977069F430E0482F552747FD509577
:103300002417350729F08595859585950C947618B1
:1033100008959091C501977081E009F480E00895C7
:1033200090910C01992321F090910D01911109C008
:1033300020910E0130910F01F90132969FEF40E08C
:103340001FC0982F9695969596959F3050F5E091D1
:103350000E01F0910F01E90FF11D877021E030E0BF
:10336000A90102C0440F551F8A95E2F7CA01918155
:10337000892B818308959F3F39F04F5F4E3041F094
:1033800051915813F8CF0DC05111F7CF942FF5CFAD
:103390009F3F39F0F901E90FF11D97FDFA958283FE
:1033A0000895089590910C01992321F090910D01B9
:1033B000911109C020910E0130910F01F90132964F
:1033C000205F3F4F1FC0982F9695969596959F30FA
:1033D000F0F4E0910E01F0910F01E90FF11D8770FB
:1033E00021E030E0A90102C0440F551F8A95E2F7A1
:1033F000CA01809591818923818308953196E217CE
:10340000F30729F090819813F9CF1082F7CF089530
:1034100081E090E0E0910E01F0910F01E80FF91FBB
:103420001082019680319105A9F708959091D901F4
:10343000892B8093D901089580959091D901892392
:103440008093D90108951092D90108959091D801DF
:10345000892B8093D801089580959091D801892374
:103460008093D80108951092D80108959091D701C2
:10347000892B8093D701089580959091D701892356
:103480008093D70108951092D70108958093C601C3
:1034900008951092C601089580910E0190910F0138
:1034A000FC0131969C01205F3F4F80E0919191118A
:1034B0008F5FE217F307D1F70895E0910E01F091C5
:1034C0000F018091D9018083E0910E01F0910F01ED
:1034D00090818091D801892B8083E0910E01F09139
:1034E0000F0190818091D701892B80838091C60143
:1034F000882361F0E0910E01F0910F019081892BFA
:1035000080830E944C1A81111092C60180910E0195
:1035100090910F010C948B0F20E0009739F0AC01D3
:1035200041505109842395232F5FF7CF822F0895AF
:10353000CF92DF92EF92FF926C01EE24FF24C11430
:10354000D104E104F10421F0C701B60120E101C07A
:1035500020E0C72ED82EE92EFF24C114D104E104A7
:10356000F10419F0285FC701B6016B017C0154E03A
:10357000F694E794D794C7945A95D1F7C114D1041F
:10358000E104F10419F02C5FC701B6016B017C0165
:1035900042E0F694E794D794C7944A95D1F7C114C2
:1035A000D104E104F10419F02E5FC701B601DC017A
:1035B000CB01B695A79597958795892B8A2B8B2B51
:1035C00009F02F5F822FFF90EF90DF90CF9008954A
:1035D0008091F101843021F11092DB0120E488E137
:1035E00090E00FB6F894A895809360000FBE2093EA
:1035F000600080E00E94780883B7817F846083BF89
:1036000083B7816083BF7894889583B78E7F83BFAB
:1036100088E10FB6F89480936000109260000FBEAE
:103620000895089508950E94111B0E94F5020E94BA
:10363000121B0E94EA0391E0811101C090E0892FE2
:1036400008950E9418140E947F0F0C94780882E05D
:1036500084BD93E095BD9AEF97BD80936E00089569
:103660002FB7F8948091DC019091DD01A091DE01EB
:10367000B091DF012FBF0895CF92DF92EF92FF92BA
:103680000F931F932FB7F8944091DC015091DD0107
:103690006091DE017091DF012FBF6A017B01EE2492
:1036A000FF248C0120E030E0C016D106E206F306CC
:1036B00010F4415051099A01281B390BC9011F917F
:1036C0000F91FF90EF90DF90CF9008951F920F928F
:1036D0000FB60F9211248F939F93AF93BF93809156
:1036E000DC019091DD01A091DE01B091DF01019636
:1036F000A11DB11D8093DC019093DD01A093DE013B
:10370000B093DF01BF91AF919F918F910F900FBE4A
:103710000F901F9018950E947C0CF8942FEF87EA69
:1037200091E6215080409040E1F700C0000087E022
:1037300090EBDC018093FB019093FC01A093FD01D1
:10374000B093FE019CE088E10FB6F894A8958093B1
:1037500060000FBE90936000FFCFEF92FF920F9337
:103760001F93CF93DF93D82FCDE08C2F0E94E303DC
:1037700005E010E0E82EF12CC701002E02C095955F
:1037800087950A94E2F780FF09C0602F7C2F80E0C4
:103790000E948805D81302C081E006C001501109BB
:1037A00058F7C15010F780E0DF91CF911F910F9132
:1037B000FF90EF900895CF93C82F8CE20E94AD1B2D
:1037C000882321F08C2FCF910C94AD1B80E0CF91FA
:1037D0000895CF930E94301D811102C00E94161DD2
:1037E000C5E6C15049F00E94F5028FE39CE90197BC
:1037F000F1F700C00000F5CF89E20E94DB1B8111C8
:1038000013C18AE20E94DB1B81110E94161D85E014
:103810000E94DB1B81110E948B1B0E943B1D809329
:10382000DA0187E00E94DB1B8823A9F18BE10E946B
:10383000DB1B882351F08091DA0181FB222720F9DC
:1038400091E0922790FB81F90EC08EE00E94DB1B75
:10385000882361F08091DA0182FB222720F991E030
:10386000922790FB82F98093DA0115C080E10E94D3
:10387000DB1B9091DA01882341F093FB222720F98A
:1038800081E0822780FB93F904C0892F809580FB1B
:1038900090F99093DA018091DA010E943F1D0E9415
:1038A0004D1D8093FA0180EE0E94DB1B882341F0BE
:1038B0008091FA01982F909590FB80F98093FA01FE
:1038C00089E30E94DB1B882359F08091FA0181FB78
:1038D000222720F991E0922790FB81F98093FA0149
:1038E00082EE0E94DB1B882359F08091FA0182FB53
:1038F000222720F991E0922790FB82F98093FA0128
:1039000086EE0E94DB1B882359F08091FA0183FB2D
:10391000222720F991E0922790FB83F98093FA0106
:1039200083EE0E94DB1B882359F08091FA0184FB0F
:10393000222720F991E0922790FB84F98093FA01E5
:1039400085E30E94DB1B882359F08091FA0185FBF7
:10395000222720F991E0922790FB85F98093FA01C4
:1039600081E30E94DB1B882359F08091FA0186FBDA
:10397000222720F991E0922790FB86F98093FA01A3
:1039800081E10E94DB1B882359F08091FA0187FBBB
:10399000222720F991E0922790FB87F98093FA0182
:1039A0008091FA010E94511D8091FA0187FB8827BE
:1039B00080F980930D0187E20E94DB1BC82F8EE106
:1039C0000E94DB1B8111C2608FE10E94DB1B811111
:1039D000C46080E20E94DB1B8111C86081E20E940A
:1039E000DB1B8111C06182E20E94DB1B8111C0627E
:1039F00083E20E94DB1B8111C06484E20E94DB1B16
:103A0000882311F0C06802C0CC2329F08C2F0E94BB
:103A1000481D6C2F03C00E94441D682F70E080E099
:103A200090E0CF910C94D817CF9108956DEE7EEF72
:103A300080E090E00E94822360E082E090E00E94BB
:103A4000702360E083E090E00E94702360E084E0F7
:103A500090E00E94702360E085E090E00C94702379
:103A600080E090E00E946A2321E08D3E9E4F09F0A5
:103A700020E0822F089582E090E00C946223682F6A
:103A800082E090E00C94702383E090E00C94622339
:103A9000682F83E090E00C94702384E090E00C9415
:103AA0006223682F84E090E00C9470238091E201FF
:103AB00080FF0BC06091130185E0689FB001112465
:103AC00075956795759567952BC081FF09C06091C5
:103AD000130185E0689FB00111247595679520C09A
:103AE00082FF07C06091130185E0689FB001112437
:103AF00017C09091E3019923D1F0609112019617BC
:103B000088F72091130185E0289F90011124929F4E
:103B1000A001939F500D112470E0CA010E9434232C
:103B20006038710540F46115710539F002C065E037
:103B300070E0862F08958FE7089581E008958091C1
:103B4000E20180FF08C06091110170E075956795F2
:103B50007595679521C081FF06C06091110170E0E5
:103B60007595679519C082FF04C06091110170E0DE
:103B700010C09091E3019923C1F060911001961754
:103B8000A0F780911101899FC001112470E00E946B
:103B900034236038710528F46115710521F0862FF2
:103BA00008958FE7089581E0089561E070E0F4CF13
:103BB000803F21F40E94561D819504C0813F29F465
:103BC0000E94561D8093E6010895823F21F40E94D1
:103BD000561D819504C0833F29F40E94561D809391
:103BE000E5010895893F19F40E949F1D05C08A3F91
:103BF00031F40E949F1D81958093E70108958B3FCA
:103C000021F40E949F1D819504C08C3F29F40E94DD
:103C10009F1D8093E8010895843F21F48091E40181
:103C2000816017C0853F21F48091E401826011C05A
:103C3000863F21F48091E40184600BC0873F21F42A
:103C40008091E401886005C0883F31F48091E401EF
:103C500080618093E40108958D3F21F48091E20119
:103C600081600BC08E3F21F48091E201826005C02B
:103C70008F3F29F48091E20184608093E2010895EE
:103C8000803F39F48091E60187FF6CC01092E60115
:103C900069C0813F29F48091E6011816BCF362C027
:103CA0009091E501823F29F497FF5CC01092E501F5
:103CB00059C0833F19F41916CCF354C0893F41F41D
:103CC0008091E70118160CF04DC01092E7014AC030
:103CD0008A3F29F48091E70187FF44C0F6CF8B3FEC
:103CE00039F48091E80187FF3DC01092E8013AC0A5
:103CF0008C3F29F48091E8011816BCF333C0843F4F
:103D000021F48091E4018E7F17C0853F21F48091DA
:103D1000E4018D7F11C0863F21F48091E4018B7F07
:103D20000BC0873F21F48091E401877F05C0883F65
:103D300031F48091E4018F7E8093E40113C08D3FC4
:103D400021F48091E2018E7F0BC08E3F21F480919F
:103D5000E2018D7F05C08F3F29F48091E2018B7FC6
:103D60008093E2018091E50181110EC08091E6010E
:103D700081110AC08091E701811106C08091E8019C
:103D8000811102C01092E301089584EE91E00E9437
:103D9000960F0E94301B9093E1018093E0010895FB
:103DA0001F93CF93DF938091E0019091E1010E94F6
:103DB0003C1BAC019091E301992321F02091140167
:103DC00030E006C0209115018AE0289F900111245F
:103DD0004217530708F486C08091E501C091E601BF
:103DE000D091E7011091E801811107C0C11176C09F
:103DF000D11174C0111172C075C09F3F19F09F5F3F
:103E00009093E301181624F40E94561D8093E50157
:103E10008091E50187FF05C00E94561D8195809322
:103E2000E5011C1624F40E94561D8093E601809142
:103E3000E60187FF05C00E94561D81958093E6012B
:103E40006091E501662339F1C091E601CC2319F1B7
:103E5000772767FD7095872F972F0E94452223E3D0
:103E600033E343E35FE30E94A9220E94122260939E
:103E7000E5016C2F772767FD7095872F972F0E949C
:103E8000452223E333E343E35FE30E94A9220E9438
:103E900012226093E6011D1624F40E949F1D809358
:103EA000E7018091E70187FF05C00E949F1D819572
:103EB0008093E701111624F40E949F1D8093E8016E
:103EC0008091E80187FF05C00E949F1D8195809326
:103ED000E801DF91CF911F910C94C51E9F3F09F01F
:103EE0008ECF96CFDF91CF911F910895E4EEF1E050
:103EF00085E0DF011D928A95E9F71092E3011092A7
:103F0000E2010895833081F128F4813059F0823044
:103F1000D1F00895853009F449C0B8F1863009F42C
:103F200056C0089580911501262F30E0280F311DCD
:103F30002F3F310524F4680F6093150108958FEF2A
:103F400080931501089580911401262F30E0280FE9
:103F5000311D2F3F310524F4680F6093140108953B
:103F60008FEF80931401089580911301262F30E084
:103F7000280F311D2F3F310524F4680F6093130182
:103F800008958FEF80931301089580911201262FD9
:103F900030E0280F311D2F3F310524F4680F609366
:103FA000120108958FEF80931201089580911101FD
:103FB000262F30E0280F311D2F3F310524F4680FE4
:103FC0006093110108958FEF8093110108958091FE
:103FD0001001262F30E0280F311D2F3F310524F42A
:103FE000680F6093100108958FEF8093100108957A
:103FF000833011F128F4813049F0823091F0089536
:10400000853081F120F18630C1F10895809115014C
:10401000681720F4861B80931501089510921501EE
:10402000089580911401681720F4861B8093140171
:10403000089510921401089580911301681720F4D7
:10404000861B8093130108951092130108958091A7
:104050001201681720F4861B8093120108951092B4
:104060001201089580911101681720F4861B809336
:10407000110108951092110108958091100168179F
:1040800020F4861B8093100108951092100108956A
:104090000F931F938D3109F46BC008F03FC08E3031
:1040A00009F47FC0C0F4873009F469C068F4863031
:1040B00009F0B1C08091DA01817F8E7F8093DA01AF
:1040C00081E08093EA01A8C0883009F4A2C08B3057
:1040D00009F49FC0A0C0863109F49BC078F48031F8
:1040E00009F472C0813109F096C00E9418149091B1
:1040F0000D0181E0892780930D018BC0893109F47E
:1041000088C08B3109F087C08091DA0181FB2227BA
:1041100020F991E0922790FB81F94CC0853309F496
:1041200070C048F4873209F46CC008F459C0893271
:1041300009F467C070C0833438F48A3308F04EC085
:10414000883309F466C067C0833409F45AC08834E0
:1041500009F061C00E9418140FEF13ED20E3015025
:1041600010402040E1F700C000000E948B1B51C0AE
:104170000E94CC210E947F0F0E9478084AC0909133
:10418000DA01892F8095817080FB90F929F0966083
:1041900098609093DA0140C0997F977F9093DA01FD
:1041A00038C08091DA0182FB222720F991E0922722
:1041B00090FB82F98093DA01992359F18091DA0119
:1041C00081608093DA0125C08091DA0183FB222788
:1041D00020F991E0922790FB83F9ECCF895301C03D
:1041E0008D5141E050E060E070E08A019B0104C025
:1041F000000F111F221F331F8A95D2F7C901B80182
:1042000004C061E070E080E090E00E94D8170E9456
:10421000181481E001C080E01F910F91089580E0A3
:10422000089580E00895CF93C82F8091EA018130EE
:1042300079F018F08230E9F187C0E0910E01F09139
:104240000F018081813169F0823209F07FC009C09D
:10425000E0910E01F0910F018081813111F08232E5
:1042600061F48C2F0E940F21811104C08C2F0E94B9
:1042700048201DC081E090E01AC08C2F0E941121BF
:10428000811114C0C43179F048F4CB3079F0C031D9
:1042900009F060C082E08093EA0108C0C93219F0D9
:1042A000C83321F057C01092EA0154C081E08170F8
:1042B00053C0C93289F118F5C43171F1A8F4C7307F
:1042C00009F046C08AE08093150194E190931401AF
:1042D00093E0909313018093120188E08093110181
:1042E00088E28093100134C0CE51C63088F5EC2F9F
:1042F000F0E0E65DFE4F80818093E90129C0CE3475
:10430000E9F020F4CB3421F56AE013C0C13579F02F
:10431000C235F1F461E00DC08091E901882319F004
:104320001092E90115C081E08093EA0115C061E0B7
:1043300006C08091E9010E94821F0AC06AE0809154
:10434000E9010E94F81F04C01092EA0180E004C055
:1043500081E002C080E0ABCFCF910895E1E8F0E0CA
:104360008081886080838081816080838FB7F894AA
:1043700093E09093890090ED909388008FBF08950B
:10438000EFE6F0E08081826080830895EFE6F0E060
:1043900080818D7F80830895EFE6F0E0908182E058
:1043A0008927808308951F920F920FB60F921124D0
:1043B0002F933F934F935F936F937F938F939F932D
:1043C000AF93BF93EF93FF938091EB019091EC013A
:1043D00001969093EC018093EB01811103C082E080
:1043E0000E947808E091EC01E695E695F0E0E85F40
:1043F000FB4FE4918091EB018E1303C080E00E949B
:104400007808FF91EF91BF91AF919F918F917F912C
:104410006F915F914F913F912F910F900FBE0F9031
:104420001F90189504D06894B1118DC0089570D074
:1044300088F09F5790F0B92F9927B751A0F0D1F08D
:10444000660F771F881F991F1AF0BA95C9F712C017
:10445000B13081F077D0B1E0089574C0672F782F24
:104460008827B85F39F0B93FCCF386957795679583
:10447000B395D9F73EF490958095709561957F4FEF
:104480008F4F9F4F0895E89409C097FB3EF4909595
:104490008095709561957F4F8F4F9F4F9923A9F01D
:1044A000F92F96E9BB279395F695879577956795AC
:1044B000B795F111F8CFFAF4BB0F11F460FF1BC0F0
:1044C0006F5F7F4F8F4F9F4F16C0882311F096E983
:1044D00011C0772321F09EE8872F762F05C0662331
:1044E00071F096E8862F70E060E02AF09A95660FEA
:1044F000771F881FDAF7880F9695879597F90895A3
:1045000057FD9058440F551F59F05F3F71F0479584
:10451000880F97FB991F61F09F3F79F08795089569
:10452000121613061406551FF2CF4695F1DF08C088
:10453000161617061806991FF1CF869571056105A5
:1045400008940895E894BB2766277727CB0197F94D
:1045500008950BD078C069D028F06ED018F095235C
:1045600009F05AC05FC01124EECFCADFA0F3959FB7
:10457000D1F3950F50E0551F629FF001729FBB274A
:10458000F00DB11D639FAA27F00DB11DAA1F649FF6
:104590006627B00DA11D661F829F2227B00DA11DA9
:1045A000621F739FB00DA11D621F839FA00D611D2F
:1045B000221F749F3327A00D611D231F849F600D50
:1045C000211D822F762F6A2F11249F5750408AF089
:1045D000E1F088234AF0EE0FFF1FBB1F661F771F15
:1045E000881F91505040A9F79E3F510570F014C0AC
:1045F000AACF5F3FECF3983EDCF3869577956795FD
:10460000B795F795E7959F5FC1F7FE2B880F911D32
:104610009695879597F9089597F99F6780E870E0D8
:1046200060E008959FEF80EC089500240A94161628
:10463000170618060906089500240A941216130690
:10464000140605060895092E0394000C11F488231E
:1046500052F0BB0F40F4BF2B11F460FF04C06F5F3A
:104660007F4F8F4F9F4F089597FB072E16F40094AE
:1046700007D077FD09D00E944E2307FC05D03EF4F9
:10468000909581959F4F0895709561957F4F0895FE
:10469000EE0FFF1F0590F491E02D0994AA1BBB1BA0
:1046A00051E107C0AA1FBB1FA617B70710F0A61B32
:1046B000B70B881F991F5A95A9F780959095BC0153
:1046C000CD010895F999FECF92BD81BDF89A992741
:1046D00080B50895A8E1B0E042E050E00C948A2350
:1046E000262FF999FECF92BD81BDF89A019700B4AB
:1046F000021639F01FBA20BD0FB6F894FA9AF99A4B
:104700000FBE08950196272F0E9471230C947023E9
:10471000DC01CB01FC01F999FECF06C0F2BDE1BD81
:10472000F89A319600B40D9241505040B8F7089570
:04473000F894FFCF2B
:1047340002207A080809E508B1087D080101C701CB
:1047440028080A03140A3F4D3639C9037C0346037B
:104754000D03A002B902D202EB0201020304050612
:044764000708090039
:00000001FF
